:020000040000FA
:1000000039EF00F0FFFFFFFF4682E1CF14F0E2CFAF
:1000100015F0D9CF16F0DACF17F0F3CF18F0F4CFF0
:1000200019F0F2AC18D00E01C0B1C8A103D04CEC4D
:1000300010F011D0C0B9C8A903D0CAEC1CF00BD085
:10004000C0BBC8AB03D00CEC19F005D0C1B7C9A731
:1000500002D020EC1EF019C0F4FF18C0F3FF17C047
:10006000DAFF16C0D9FF15C0E2FF14C0E1FF4692C7
:10007000110059EF18F0FFFFFFFFFFFFFFFFFFFF29
:10008000FFFFFFFFFFFFFFFFFFFFFFFFFFFFFFFF80
:10009000FFFFFFFFFFFFFFFFFFFFFFFFFFFFFFFF70
:1000A000FFFFFFFFFFFFFFFFFFFFFFFFFFFFFFFF60
:1000B000FFFFFFFFFFFFFFFFFFFFFFFFFFFFFFFF50
:100800000043445A207C20207C20207C20207C2017
:1008100020004E6F7468616C742C204164722E202D
:1008200034390020202020202020202020202020BB
:1008300020007374726F6D207A7520686F63682171
:10084000004261747465726965204C6164652D00B5
:100850004344462D53657475703A204265690048DB
:1008600052582D496E746572666163650043445A3F
:1008700020485220202020202000205761727465DB
:100880002061756620004C6164656E20302C20204C
:10089000410048525820636F6E6E65637400467560
:1008A0006E6B2D5363616E0056657273696F6E20B7
:1008B0000043445A20485200485220203A00434402
:1008C0005A2000000201916FE3D2D3EC18F012001D
:1008D0000001FA51D8A40DD076EC1DF09E0E1E6ECC
:1008E0000A0E1F6E02EC1AF0010E1E6E020E05ECCF
:1008F0001CF00001FA51990FD96EDA6ADF50D8B4B2
:100900001200020EF06FFA51030DF3CFF1F0FA511D
:100910009F0FD96EDA6ADF503BEC1BF01200CC0E51
:100920000001FA25D96EDA6A010EDA22DF500201DF
:10093000966F0001F905D8A430D076EC1DF0B10E09
:100940001E6E070E1F6E02EC1AF00001FC05D8A403
:100950000CD0050E1E6E020E05EC1CF0860E1E6EEF
:100960000C0E1F6E02EC1AF018D0020E020196193E
:10097000D8A413D00001FA51990FD96EDA6ADF506A
:10098000D8B40BD0050E1E6E020E05EC1CF0710ED5
:100990001E6E090E1F6E02EC1AF00001FB05D8A4B2
:1009A00032D0050E1E6E0201965105EC1CF00201BC
:1009B0009605D8A41DD076EC1DF0010E1E6E010E1A
:1009C00005EC1CF06D0E1E6E0D0E1F6E02EC1AF083
:1009D0000001FC05D8A41200050E1E6E020E05ECE7
:1009E0001CF0860E1E6E0C0E1F6E02EC1AF012002A
:1009F0000001FC51D8A41200230E1E6E0F0E1F6EB4
:100A000002EC1AF01200FA510E0D010EF324D96E09
:100A1000020EF420DA6EDF500201956F0001FA51E8
:100A20000E0D020EF324D96E020EF420DA6EDF50A2
:100A30000201946F0001FA510E0D030EF324D96EDA
:100A4000020EF420DA6E0201DFAC02D0010E01D0FA
:100A5000000E926F0001FA510E0D030EF324D96EB1
:100A6000020EF420DA6E0201DFAA02D0010E01D0DC
:100A7000000E906F0001FA510E0D030EF324D96E93
:100A8000020EF420DA6E0201DFA403D095513D0F6F
:100A9000956F9605D8A445D0050E1E6E010E05EC87
:100AA0001CF095C2EFF094C2F0F0000E0001F16F5F
:100AB000000EF26F92C2F3F0000EF46F96C2F5F0E2
:100AC000070EF66F010EF76FFA51B8EC16F0000141
:100AD000F905D8A40FD0FC51D8A40CD0050E1E6E79
:100AE000020E05EC1CF0250E1E6E0D0E1F6E02ECA4
:100AF0001AF01200FC05D8A41200B0EC1CF00D0E88
:100B00001E6E020E05EC1CF0010E1A6E2C50300FFA
:100B1000A7EC1AF0010E1A6E2A50300FA7EC1AF04B
:100B200012000001FC51D8A41200FA51990FD96E9D
:100B3000DA6ADF50D8B41200050E1E6E020E05EC04
:100B40001CF0B50E1E6E030E1F6E02EC1AF095C25D
:100B5000EFF094C2F0F0000E0001F16F000EF26FA2
:100B600092C2F3F0000EF46F96C2F5F0070EF66F26
:100B7000010EF76FFA51B8EC16F01200060E05D010
:100B8000090E03D00C0E01D00F0E0201936F0FD08F
:100B90000001FA51010AD8B4F1D7030AD8B4F0D74A
:100BA000010AD8B4EFD7070AD8B4EED7E7D70001C7
:100BB000F905D8A475D076EC1DF0010E1E6E110E4D
:100BC0001F6E02EC1AF0050E1E6E010E05EC1CF0F5
:100BD000010E1A6E000EA7EC1AF02F0E1E6E030EF9
:100BE0001F6E02EC1AF0010E1A6E000EA7EC1AF03E
:100BF0002F0E1E6E030E1F6E02EC1AF0010E1A6EFF
:100C0000000EA7EC1AF02F0E1E6E030E1F6E02ECE4
:100C10001AF0010E1A6E000EA7EC1AF02F0E1E6EBF
:100C2000030E1F6E02EC1AF0050E1E6E020E05EC8E
:100C30001CF00001FC05D8A407D0860E1E6E0C0E19
:100C40001F6E02EC1AF02CD0010E1A6E000EA7ECEB
:100C50001AF02F0E1E6E030E1F6E02EC1AF0010E1C
:100C60001A6E000EA7EC1AF02F0E1E6E030E1F6EEA
:100C700002EC1AF0010E1A6E000EA7EC1AF02F0EFD
:100C80001E6E030E1F6E02EC1AF0010E1A6E000E9D
:100C9000A7EC1AF02F0E1E6E030E1F6E02EC1AF058
:100CA0000001FB05D8A40CD093C21EF0010E05EC88
:100CB0001CF02F0E1E6E030E1F6E02EC1AF01200B7
:100CC000FA510E0D010EF324D96E020EF420DA6EE5
:100CD000DF500201956F0001FA510E0D020EF32450
:100CE000D96E020EF420DA6EDF500201946F00011B
:100CF000FA510E0D030EF324D96E020EF420DA6EB3
:100D00000201DFA403D095513D0F956F93C21EF0F1
:100D1000010E05EC1CF002019551C4EC1BF0000122
:100D2000FC05D8A414D0B0EC1CF00D0E1E6E020E03
:100D300005EC1CF0010E1A6E2C50300FA7EC1AF0C7
:100D4000010E1A6E2A50300FA7EC1AF01200FA5159
:100D5000990FD96EDA6ADF50D8B4120002019305F8
:100D60001E6E020E05EC1CF0020194A506D0010EC9
:100D70001A6E010EA7EC1AF005D0010E1A6E000EC5
:100D8000A7EC1AF002019439E8461F0BC4EC1BF0E3
:100D90001200050E1E6E020E05EC1CF00001BE5185
:100DA000D8A406D0860E1E6E0C0E1F6E02EC1AF032
:100DB000B0EC1CF00D0E1E6E020E05EC1CF0010EC8
:100DC0001A6E2C50300FA7EC1AF0010E1A6E2A5032
:100DD000300FA7EC1AF0010E0001BE6F12000001E7
:100DE000F905D8B476EC1DF0030E1E6E010E05EC6D
:100DF0001CF0410E1E6E0F0E1F6E02EC1AF0030E59
:100E00001E6E020E05EC1CF0320E1E6E0F0E1F6ED3
:100E100002EC1AF01200020E0001F06F090EF16FE1
:100E200035503BEC1BF0020E0001F06F090EF16F24
:100E300035503BEC1BF01200010E1E6E010E05EC4E
:100E40001CF0BE0E1E6E050E1F6E02EC1AF0B80EE0
:100E50001E6E060E1F6E02EC1AF01200050E1E6EBC
:100E6000010E05EC1CF07A0E1E6E0C0E1F6E02ECCD
:100E70001AF0050E1E6E020E05EC1CF0920E1E6E90
:100E80000C0E1F6E02EC1AF0120018EC1BF0120090
:100E900002019151010AD8B418D5030AD8B418D563
:100EA000010AD8B43CD5070AD8B472D6010AD8B41E
:100EB0000CD5030AD8B46DD7010AD8B490D70F0A5D
:100EC000D8B4A9D7010AD8B4B7D7030AD8B4C6D7BB
:100ED000010AD8A41200D9D7246E0F0E286E245010
:100EE000D8B40FD0010E266E26509F0FD96EDA6A45
:100EF0002450DE18D8B426C028F0262A040E266412
:100F0000F3D70F0E2818D8A44ED29BD22850990F91
:100F1000D96EDA6ADFB012D028509F0FD96EDA6A24
:100F2000000E2824E16EE26A020EE222DFCFE7FF24
:100F30002850990FD96EDA6A000EDB80B40E28248F
:100F4000D96EDA6A010EDA2266C0DFFF130E62651F
:100F500002D0130E626F0D0E676502D00D0E626F28
:100F600062C025F02550620FD96EDA6ABA0E2824C5
:100F7000E16EE26A010EE222DFCFE7FF28500E0D9C
:100F8000000EF324D96E020EF420DA6E67C0DFFF84
:100F9000010E276E35D02750670FD96EDA6A2850B8
:100FA0000E0D000E216E020E226EF3502126F4501B
:100FB000222227502124E16E000E2220E26EDE5014
:100FC000E618D8B41CD02750670FD96EDA6A2850BB
:100FD0000E0D000E206E020E216EF3502026F450EE
:100FE000212227502024E16E000E2120E26EDFCF67
:100FF000E7FF2850990FD96EDA6A000EDB82272AA4
:1010000028500E0D000EF324D96E020EF420DA6E75
:101010002750DE5CD8B0BFD72850870FD96EDA6A68
:101020006CC0DFFFAE0E2824D96EDA6A010EDA2218
:101030006DC0DFFFAE0E2824D96EDA6A010EDA2207
:101040000101DFA29CD028500E0D010EF324D96EB1
:10105000020EF420DA6EDF503F0B310AD8A48FD095
:1010600028500E0D030EF324D96E020EF420DA6E12
:101070000201DFA884D034A003D0206A202A01D046
:10108000206A34A202D0010E01D0000E020DF3CF6F
:1010900021F034A402D0010E01D0000E040DF35053
:1010A00021242024256E28500E0D020EF324D96E23
:1010B000020EF420DA6EDF50206ED8902032D890E5
:1010C0002032D89020302518D8B459D028500E0D91
:1010D000020EF324D96E020EF420DA6EDF50206E79
:1010E000D8902032D8902032D8902032010E20168D
:1010F00034502018FE0B2018346E28500E0D020EAE
:10110000F324D96E020EF420DA6EDF50206E203AFE
:101110000F0E2016010E2016204634502018FD0B0D
:101120002018346E28500E0D020EF324D96E020ED4
:10113000F420DA6EDF50206E050E216ED89020323A
:10114000212EFCD7010E20162046204634502018B0
:10115000FB0B2018346E0F0E1D6E28500E0D020E64
:10116000F324D96E020EF420DA6EDF50206ED89090
:101170002032D8902032D8902030E4EC1CF0370494
:10118000D8A444D0AE0E2824D96EDA6A010EDA2231
:101190000101DFA611D03150D8A40ED0AE0E282404
:1011A000D96EDA6A010EDA22F00EDF1628507B0FB4
:1011B000D96EDA6AF00EDF16AE0E2824D96EDA6A1E
:1011C000010EDA22DFA00BD03150D8A408D08484DD
:1011D00028507B0FD96EDA6A060EDF125ED0AE0E93
:1011E0002824D96EDA6A010EDA22DFA656D02850FA
:1011F0007B0FD96EDA6A0001DFA44FD084942850A7
:101200007B0FD96EDA6A000EDB8447D0AE0E28243D
:10121000D96EDA6A010EDA220101DFA612D031504E
:10122000D8A40FD0AE0E2824D96EDA6A010EDA22C5
:10123000F00EDF1628507B0FD96EDA6AF00EDF163B
:101240008494AE0E2824D96EDA6A010EDA22DFA069
:101250000CD03150D8A409D0848428507B0FD96E8B
:10126000DA6A060EDF12010E17D0AE0E2824D96EF0
:10127000DA6A010EDA22DFA610D028507B0FD96E71
:10128000DA6A0001DFA409D0849428507B0FD96E5C
:10129000DA6A000EDB84000E316E2850990FD96E89
:1012A000DA6A7F0EDF1628509F0FD96EDA6A530E66
:1012B0002824E16EE26A010EE222DFCFE7FF89D047
:1012C0002850990FD96EDA6A010EDF6EECD764519F
:1012D000D8A402D0010E01D0000E206E6351D8A414
:1012E00002D0010E01D0000E2014E8A072D00F0E23
:1012F0003D18D8B46ED03D50D8B46BD03DC028F066
:101300002850990FD96EDA6A000EDB88080E3E6EFF
:1013100028508D0FD96EDA6A000EDF6E06D0285085
:101320008D0FD96EDA6AB4CFDFFF28508D0FD96EDA
:10133000DA6ADF50D8B4F3D7C00E2824D96EDA6A3F
:10134000010EDA222F0EDF6E44D03DC028F0285067
:101350009F0FD96EDA6ADE506319D8A421D02850C5
:101360008D0FD96EDA6ADE506419D8A419D02850CE
:10137000990FD96EDA6A010EDF6EC60E2824D96E77
:10138000DA6A010EDA22000EDF6E28508D0FD96E58
:10139000DA6ADF501D6E285023EC1CF0000E3E6E02
:1013A000000E3D6E16D000016551BF0B206E216A04
:1013B0002150000AD8A40DD02050300AD8B480D7CC
:1013C000010AD8B4A3D50F0AD8B481D7010AD8B47A
:1013D000BCD7285012006451D8A402D0010E01D00D
:1013E000000E206E6351D8A402D0010E01D0000E71
:1013F0002014E8A0EED70F0E3D18D8B4EAD73D5020
:10140000D8B4E7D73DC028F02850990FD96EDA6AD2
:10141000000EDB88080E3E6E28508D0FD96EDA6AFA
:10142000000EDF6E06D028508D0FD96EDA6AB4CF69
:10143000DFFF28508D0FD96EDA6ADF50D8A47CD731
:10144000F2D700016551BF0B206E216A2150000ABE
:10145000D8A4BFD72050300AD8B432D70E0AD8B497
:10146000BAD7B7D788EC1DF0F28EF28C829096EC4A
:1014700018F00E0EF2EC1DF05A0AD8A415D00F0E7B
:10148000F2EC1DF002019B6F9BB134800F0EF2EC69
:101490001DF002019B6F9BB334820F0EF2EC1DF026
:1014A00002019B6F9BB5348477EC13F0010E0001B1
:1014B000F96F010EFA6F000EFB6F000EFC6F010E4C
:1014C00062EC04F0520E02019C6F2B0E9B6F000E1B
:1014D000E82EFED79B2FFCD79C2FFAD700F0010EE9
:1014E0000001F96F010EFA6F000EFB6F000EFC6F2A
:1014F0000B0E62EC04F07A0E02019C6FC10E9B6F22
:10150000810EE82EFED79B2FFCD79C2FFAD700D058
:10151000828027EC1EF025EC1EF0410E02019C6F2C
:10152000F00E9B6F330EE82EFED79B2FFCD79C2F1F
:10153000FAD7000E0001F96F000EFA6F000EFB6F74
:10154000000EFC6F020E62EC04F0190E02019C6F9B
:101550005A0E9B6FB10EE82EFED79B2FFCD79C2F07
:10156000FAD700D0010E0001B26F010E0201A06F88
:10157000A0518D0FD96EDA6ADF50D8B45DD0A0517A
:101580008D0FD96EDA6ADF50246E210E256E000EA3
:10159000266EA0519F0FD96EDA6ADF503CEC14F032
:1015A000FA0E02019B6F580EE82EFED79B2FFCD738
:1015B00000F00001D705D8A43FD0400E6119D8A48F
:1015C0000BD0000ED76FFA0E02019B6F580EE82E5B
:1015D000FED79B2FFCD700F0810E00016119D8A423
:1015E0001ED0000ED76FD3EC17F0B62B0201A0511E
:1015F0009F0FD96EDA6AA20E0001B625E16EE26A8B
:10160000010EE222DFCFE7FF000EF96FA0C2FAF071
:10161000000EFB6F000EFC6F020E62EC04F0190E60
:1016200002019C6F5A0E9B6FB10EE82EFED79B2FC6
:10163000FCD79C2FFAD700D00201A02B040EA06586
:1016400097D7410E02019C6FF00E9B6F330EE82E70
:10165000FED79B2FFCD79C2FFAD7000E0001B26F4C
:10166000010EBC6F000E3D6E000E396EBBEC1DF01E
:1016700076EC1DF0010E0001F96F010EFA6F000EFD
:10168000FB6F000EFC6F090E62EC04F0090E336E66
:10169000F5EC1AF00001AB51D8A425D0990EAB6F30
:1016A000000E3E6E3D50D8B412D03D50990FD96E09
:1016B000DA6ADFB00CD03D50990FD96EDA6A000EAD
:1016C000DF6E3D50810FD96EDA6A000EDF6EE6ECF8
:1016D0001DF03D6E0F0E3D18D8B403D0040E3E6EC3
:1016E00002D0000E3D6E0001D705D8A40DD0D3EC7A
:1016F00017F002019D6F000E0001D76F220E216EC0
:1017000002019D5191EC12F00001CD51D8A415D0E9
:10171000990ECD6F000E396E010E02019E6F040E00
:101720009E6501D00AD0DE0E9E25D96EDA6A010EC2
:10173000DA22000EDF6E9E2BF2D73950D8A449D0A2
:101740000001B051D8A445D0030EB06F040E3A6426
:1017500003D0010E3A6E01D03A2A3E50D8B422D0BE
:101760003EA612D03D508D0FD96EDA6ADF50246E3E
:101770002F0E256E000E266E3D509F0FD96EDA6A31
:10178000DF503CEC14F00BD03EA409D0000E246EC8
:101790002E0E256E000E266E000E3CEC14F0000E90
:1017A0003E6E17D03A50D8B414D03A508D0FD96E3F
:1017B000DA6ADF50D8B40DD03A500C0D540EF32431
:1017C000D96E020EF420DA6E000EDF6E3A50C2ECD3
:1017D00015F0000E2F6E010E0201A36F040EA3651B
:1017E00001D03BD0A351750FD96EDA6A070EDF64C2
:1017F00020D0A351750FD96EDA6A000EDF6E530E3A
:10180000A325D96EDA6A010EDA22000EDF6EA3512B
:10181000990FD96EDA6A000EDF6EA351870FD96E69
:10182000DA6A000EDF6EA351810FD96EDA6A000EFC
:10183000DF6EA351990FD96EDA6A0001DFA00AD0DA
:101840002F2ACC0E0201A325D96EDA6A010EDA2204
:101850002FC0DFFF0201A32BC1D70001AF51D8A4D5
:1018600004D01E0EAF6F81EC1BF00001AE51D8A466
:101870000FD70A0EAE6F000E0201976F0001AA513A
:101880007EEC11F00001AA2B050EAA19D8A400D7EE
:10189000010EAA6F030E63EC1DF01AC0A1F21BC06B
:1018A000A2F20201A2A103D0000EA26FA169A2A31D
:1018B00004D0000EA26F000EA16F0001DF2B070EF7
:1018C000DF6502D0000EDF6F990EDF25D96EDA6A70
:1018D000010EDA22A1C2DFFF000E0201A26F000E8C
:1018E000A16F000E9F6F070E9F6501D00ED0990E5D
:1018F0009F25D96EDA6A010EDA22DF509B6F9B5169
:10190000A127000EA2239F2BEED7A1C29BF2A2C259
:101910009CF2D8909C339B33D8909C339B33D890C7
:101920009C339B339B51366E050E63EC1DF01AC041
:10193000A1F21BC0A2F2A1C21AF0A2C21BF0000EBB
:101940001D6E0E0E1C6E56EC1AF01A50356E040EFB
:1019500063EC1DF01AC0A1F21BC0A2F2A1C21AF0E2
:10196000A2C21BF0000E1D6E1B0E1C6E56EC1AF070
:101970001A500001B46F8CD6216EBBD121500C0DD2
:10198000540EF324D96E020EF420DA6EDF50206E6E
:1019900021500E0D000EF324D96E010EF420DA6EE4
:1019A000060EDF6E2150930FD96EDA6ADF501B6E80
:1019B000030E1B162150870FD96EDA6ADF50030B16
:1019C0001B18D8A4EDD02150930FD96EDA6A21509C
:1019D000810FE16EE26ADFCFE7FF20AE06D0215033
:1019E000810FD96EDA6A000EDB8E2150870FD96E17
:1019F000DA6A0001DFB83FD020BA13D021500E0DB3
:101A0000010EF324D96E020EF420DA6E21500E0D71
:101A1000010EF324E16E010EF420E26EDFCFE7FF4A
:101A20000AD021500E0D010EF324D96E010EF420C0
:101A3000DA6E000EDF6E20B813D021500E0D040EAA
:101A4000F324D96E020EF420DA6E21500E0D040E2E
:101A5000F324E16E010EF420E26EDFCFE7FF2FD01A
:101A600021500E0D040EF324D96E010EF420DA6E0F
:101A7000000EDF6E24D021500E0D010EF324D96E1E
:101A8000020EF420DA6E21500E0D010EF324E16EE9
:101A9000010EF420E26EDFCFE7FF2150930FD96EE5
:101AA000DA6A2150810FE16EE26ADFCFE7FF20AEF4
:101AB000D7D72150810FD96EDA6A000EDB8E215004
:101AC000870FD96EDA6ADFAA10D02150930FD96E32
:101AD000DA6A2150810FE16EE26ADFCFE7FF215021
:101AE000810FD96EDA6A000EDB8E2150870FD96E16
:101AF000DA6ADFAC10D02150930FD96EDA6A215028
:101B0000810FE16EE26ADFCFE7FF2150810FD96ECE
:101B1000DA6A000EDB8E21500E0D030EF324D96E0F
:101B2000010EF420DA6E0101DFAC11D02150990FC3
:101B3000D96EDA6A000EDB8C21500E0D010EF324F3
:101B4000D96E010EF420DA6E000EDB8C06D0215027
:101B5000990FD96EDA6ABF0EDF1621500E0D020EF4
:101B6000F324D96E020EF420DA6E21500E0D020E0F
:101B7000F324E16E010EF420E26EDFCFE7FF215087
:101B80000E0D030EF324D96E020EF420DA6E2150EE
:101B90000E0D030EF324E16E010EF420E26E4BD025
:101BA00021500E0D010EF324D96E020EF420DA6ED0
:101BB00021500E0D010EF324E16E010EF420E26EB1
:101BC000DFCFE7FF21500E0D020EF324D96E020E77
:101BD000F420DA6E21500E0D020EF324E16E010E98
:101BE000F420E26EDFCFE7FF21500E0D030EF32449
:101BF000D96E010EF420DA6E21500E0D030EF3247F
:101C0000E16E020EF420E26EE750040BDF6E21500D
:101C10000E0D040EF324D96E010EF420DA6E000EC0
:101C2000DF6E2150930FD96EDA6A000EDB822150ED
:101C3000810FE16EE26ADFCFE7FF3704D8A413D04B
:101C400020B609D0000E316E21507B0FD96EDA6AB2
:101C5000FD0EDF1608D0010E316E21507B0FD96EBC
:101C6000DA6A000EDB822150810FD96EDA6A2150C8
:101C70000E0D050EF324E16E010EF420E26EDFCFAF
:101C8000E7FF21507B0FD96EDA6A21500E0D060E48
:101C9000F324E16E010EF420E26EDFCFE7FF1200C5
:101CA000010E1F6E21500E0D000E1B6E020E1C6EDB
:101CB000F3501B26F4501C221F501B24D96E000E1B
:101CC0001C20DA6E21500E0D000E1D6E010E1E6ED0
:101CD000F3501D26F4501E221F501D24E16E000EED
:101CE0001E20E26EDFCFE7FF1F2A060E1F64DAD741
:101CF00012001A50230AD8B441D60B0AD8B41200E5
:101D00004B0AD8A41200CCD7086EBBD108500C0DDA
:101D1000540EF324D96E020EF420DA6EDF50076EF3
:101D200008500E0D000EF324D96E010EF420DA6E69
:101D3000060EDF6E0850930FD96EDA6ADF50026E1E
:101D4000030E02160850870FD96EDA6ADF50030BB4
:101D50000218D8A4EDD00850930FD96EDA6A085053
:101D6000810FE16EE26ADFCFE7FF07AE06D00850D1
:101D7000810FD96EDA6A000EDB8E0850870FD96E9C
:101D8000DA6A0001DFB83FD007BA13D008500E0D51
:101D9000010EF324D96E020EF420DA6E08500E0DF7
:101DA000010EF324E16E010EF420E26EDFCFE7FFB7
:101DB0000AD008500E0D010EF324D96E010EF42046
:101DC000DA6E000EDF6E07B813D008500E0D040E49
:101DD000F324D96E020EF420DA6E08500E0D040EB4
:101DE000F324E16E010EF420E26EDFCFE7FF2FD087
:101DF00008500E0D040EF324D96E010EF420DA6E95
:101E0000000EDF6E24D008500E0D010EF324D96EA3
:101E1000020EF420DA6E08500E0D010EF324E16E6E
:101E2000010EF420E26EDFCFE7FF0850930FD96E6A
:101E3000DA6A0850810FE16EE26ADFCFE7FF07AE92
:101E4000D7D70850810FD96EDA6A000EDB8E0850A2
:101E5000870FD96EDA6ADFAA10D00850930FD96EB7
:101E6000DA6A0850810FE16EE26ADFCFE7FF0850BF
:101E7000810FD96EDA6A000EDB8E0850870FD96E9B
:101E8000DA6ADFAC10D00850930FD96EDA6A0850C6
:101E9000810FE16EE26ADFCFE7FF0850810FD96E54
:101EA000DA6A000EDB8E08500E0D030EF324D96E95
:101EB000010EF420DA6E0101DFAC11D00850990F49
:101EC000D96EDA6A000EDB8C08500E0D010EF32479
:101ED000D96E010EF420DA6E000EDB8C06D00850AD
:101EE000990FD96EDA6ABF0EDF1608500E0D020E7A
:101EF000F324D96E020EF420DA6E08500E0D020E95
:101F0000F324E16E010EF420E26EDFCFE7FF08500C
:101F10000E0D030EF324D96E020EF420DA6E085073
:101F20000E0D030EF324E16E010EF420E26E4BD091
:101F300008500E0D010EF324D96E020EF420DA6E55
:101F400008500E0D010EF324E16E010EF420E26E36
:101F5000DFCFE7FF08500E0D020EF324D96E020EFC
:101F6000F420DA6E08500E0D020EF324E16E010E1D
:101F7000F420E26EDFCFE7FF08500E0D030EF324CE
:101F8000D96E010EF420DA6E08500E0D030EF32404
:101F9000E16E020EF420E26EE750040BDF6E085093
:101FA0000E0D040EF324D96E010EF420DA6E000E2D
:101FB000DF6E0850930FD96EDA6A000EDB8208508C
:101FC000810FE16EE26ADFCFE7FF3704D8A413D0B8
:101FD00007B609D0000E316E08507B0FD96EDA6A51
:101FE000FD0EDF1608D0010E316E08507B0FD96E42
:101FF000DA6A000EDB820850810FD96EDA6A085067
:102000000E0D050EF324E16E010EF420E26EDFCF1B
:10201000E7FF08507B0FD96EDA6A08500E0D060EE6
:10202000F324E16E010EF420E26EDFCFE7FF120031
:10203000010E066E08500E0D000E026E020E036EAB
:10204000F3500226F450032206500224D96E000EEB
:102050000320DA6E08500E0D000E046E010E056EA0
:10206000F3500426F450052206500424E16E000EBD
:102070000520E26EDFCFE7FF062A060E0664DAD7F8
:1020800012000150230AD8B441D60B0AD8B412006A
:102090004B0AD8A41200CCD7C89194A442D091CFB7
:1020A00013F03B50D8A424D0D8901330136E1350A3
:1020B0000001A019D8A402D0010E13D01350A11909
:1020C000D8A402D0020E0DD01350A219D8A402D069
:1020D000030E07D01350A319D8A402D0040E01D0C8
:1020E000000E3A6E010E386E39508109396E3998FA
:1020F00094AA02D096BC5AD03A500C0D540E116ED0
:10210000010E126EF3501126F45012223B5011248E
:10211000D96E000E1220DA6EDF50916E3B2A398C98
:1021200045D094BA25D091CF13F0D8901330136EC8
:10213000000E3B6E13500001A019D8A402D0010E6E
:1021400013D01350A119D8A402D0020E0DD01350F1
:10215000A219D8A402D0030E07D01350A319D8A4F3
:1021600002D0040E01D0000E3A6E010ECB6F1ED0CD
:1021700094B81CD091CF13F03A500C0D540E116E40
:10218000020E126EF3501126F45012223B5011240D
:10219000D96E000E1220DA6E13C0DFFF3B2A3BC05F
:1021A000CEF0010E376E990E0001CD6F9588978C99
:1021B000000E0001CC6F94A81200979C000E3B6E9D
:1021C000010ECC6F3804D8A420D03F0E3916398ABE
:1021D000000E386E3A50990FD96EDA6ADFA206D037
:1021E0003A50990FD96EDA6A000EDB8ED20E3A247D
:1021F000D96EDA6A010EDA22D80E3A24E16EE26A6A
:10220000010EE222DFCFE7FF1200CB05D8A41200B7
:10221000399A3988000ECB6FD80E3A24D96EDA6A13
:10222000010EDA223A50930FE16EE26ADFCFE7FF48
:102230003E50D8B422D03EA612D03D508D0FD96E5C
:10224000DA6ADF500B6E2F0E0C6E000E0D6E3D50D5
:102250009F0FD96EDA6ADF50FFEC14F00BD03EA46A
:1022600009D0000E0B6E2E0E0C6E000E0D6E000EC1
:10227000FFEC14F0000E3E6E12003A50D8A412D0BB
:10228000040E3C6403D0010E3C6E01D03C2A3C504D
:102290008D0FD96EDA6ADF50D8B412003C503DEC95
:1022A00016F012003A50990FD96EDA6ADF50820B9D
:1022B000820AD8A411D03A50990FD96EDA6A7D0EED
:1022C000DF163A508D0FD96EDA6ADF50D8B412009B
:1022D0003A503DEC16F01200040E3C6403D0010E9F
:1022E0003C6E01D03C2A3C508D0FD96EDA6ADF502B
:1022F000D8B412003C503DEC16F0120002019A6F67
:10230000000E0201986F34A210D01C0E366405D066
:102310002E50D8A40CD0010E04D02E04D8A407D07F
:10232000000E2E6E010E986F02D0000E2E6E760EED
:10233000366415D034A213D0070E3318D8B4120067
:10234000010E0001F96F9AC2FAF0000EFB6F020E47
:10235000FC6F070E62EC04F0070E336E1200720E73
:10236000366006D0070E3318D8A402D0010E986F3D
:10237000020E2F6464D0040E3318D8B405D0010EB9
:10238000996F040E336E02D0000E996F9A51990F17
:10239000D96EDA6ADF50D8A429D0C60E9A25D96E34
:1023A000DA6A010EDA22DF50D8A420D0C60E9A25B0
:1023B000D96EDA6A010EDA22010EDF6E99C2F9F0E7
:1023C0009AC2FAF0010E0001FB6F2EC0FCF03350F0
:1023D00062EC04F0CC0E02019A25D96EDA6A010E85
:1023E000DA22000EDF6E000E2E6E12009A51990F47
:1023F000D96EDA6ADF50D8B412D09805D8A402D0CA
:10240000010E996F99C2F9F09AC2FAF0000E00011C
:10241000FB6F2EC0FCF0335062EC04F01200990503
:10242000D8A41200010E0001F96F9AC2FAF0000E52
:10243000FB6F2EC0FCF0335062EC04F012002F5002
:10244000D8B459D0030E3318D8B405D0010E996F03
:10245000030E336E02D0000E996F9A51990FD96E08
:10246000DA6ADF50D8A41ED0C60E9A25D96EDA6A71
:10247000010EDA22DF50D8A415D0C60E9A25D96EE7
:10248000DA6A010EDA22010EDF6E99C2F9F09AC201
:10249000FAF0010E0001FB6F2EC0FCF0335062EC2D
:1024A00004F098D79A51990FD96EDA6ADF50D8B4F0
:1024B00012D09805D8A402D0010E996F99C2F9F0F4
:1024C0009AC2FAF0000E0001FB6F2EC0FCF03350F0
:1024D00062EC04F012009905D8A41200010E00016C
:1024E000F96F9AC2FAF0000EFB6F2EC0FCF0335069
:1024F00062EC04F012002F50D8A412000A0E331818
:10250000D8B412000A0E336E010E0001F96F9AC2A0
:10251000FAF0000EFB6F2EC0FCF0335062EC04F0BA
:102520001200256E000E246EDCD02550D8B49AD04F
:1025300025500E0D010EF324D96E020EF420DA6E32
:10254000DF500101906F25500E0D020EF324D96E5D
:10255000020EF420DA6EDF50FC0B916F25500C0D4B
:10256000550EF324D96E010EF420DA6EDF50226E80
:10257000FC0E221625500E0D020EF324D96E020E0B
:10258000F420DA6EDF50FC0B2218D8A4918325507A
:102590000E0D030EF324D96E020EF420DA6EDF5016
:1025A000926F25500C0D560EF324D96E010EF420B7
:1025B000DA6E25500E0D030EF324E16E020EF420A8
:1025C000E26EDE50E618D8B40DD025500E0D030E85
:1025D000F324D96E020EF420DA6E0201DFBE02D0BF
:1025E0000101918125500E0D040EF324D96E020EC7
:1025F000F420DA6EDF500101936F25500C0D540E5C
:10260000F324D96E010EF420DA6E90C1DFFF25505D
:102610000C0D550EF324D96E010EF420DA6E91C123
:10262000DFFF25500C0D560EF324D96E010EF42059
:10263000DA6E92C1DFFF25500C0D570EF324D96ED0
:10264000010EF420DA6E93C1DFFF2550870FD96E9B
:10265000DA6AD20E2524E16EE26A010EE222DFCFB1
:10266000E7FF120000019A51D8A404D0000E010126
:10267000906F05D0490E0101906F050E246E000188
:102680009B51D8A404D0000E0101916F05D04A0ED1
:102690000101916F060E246E00019C51D8A404D054
:1026A000000E0101926F05D04B0E0101926F070ED3
:1026B000246E00019D51D8A404D0000E0101936F37
:1026C00005D04C0E0101936F080E246E2450060FA6
:1026D0001E6E020E05EC1CF02450300F09EC1EF0AB
:1026E00012002150220AD8B420D7010A1200090E84
:1026F0001F6E1E0E1E6EE40EE82EFED71E2EFCD799
:102700001F2EFAD700D0000E1A6E380E2CEC1AF0DD
:10271000B60E00D000D0E82EFCD700D000D000D0FC
:10272000000E1A6E380E2CEC1AF0B60E00D000D047
:10273000E82EFCD700D000D000D0010E1A6E0C0E8F
:102740002CEC1AF0B60E00D000D0E82EFCD700D04A
:1027500000D000D0010E1A6E010E2CEC1AF02A0ED9
:102760001E6E8E0EE82EFED71E2EFCD7010E1A6EA0
:10277000060E2CEC1AF02A0E1E6E8E0EE82EFED7D8
:102780001E2EFCD7010E1A6E020E2CEC1AF02A0E29
:102790001E6E8E0EE82EFED71E2EFCD7010E1A6E70
:1027A000400E2CEC1AF0010E1A6E080EA7EC1AF06F
:1027B000010E1A6E080EA7EC1AF0010E1A6E080E22
:1027C000A7EC1AF0010E1A6E080EA7EC1AF0010E13
:1027D0001A6E080EA7EC1AF0010E1A6E080EA7EC7E
:1027E0001AF0010E1A6E080EA7EC1AF0010E1A6EFE
:1027F000080EA7EC1AF0010E1A6E480E2CEC1AF017
:10280000010E1A6E080EA7EC1AF0010E1A6E080ED1
:10281000A7EC1AF0010E1A6E080EA7EC1AF0010EC2
:102820001A6E0A0EA7EC1AF0010E1A6E0B0EA7EC28
:102830001AF0010E1A6E0A0EA7EC1AF0010E1A6EAB
:102840000A0EA7EC1AF0010E1A6E080EA7EC1AF089
:102850002A0E1E6E8E0EE82EFED71E2EFCD7010EFF
:102860001A6E020E2CEC1AF02A0E1E6E8E0EE82E38
:10287000FED71E2EFCD71200286E24C01AF0285056
:102880005DEC1CF0296E259CAFD028C0E0F024C080
:10289000E1F0210E0001E26F3104D8B4E28D26C0D0
:1028A000E3F0000EE46F050E306E0F0E2918D8B459
:1028B00046D0230E1A6E2950BCEC0CF0060E000117
:1028C000E46F29500E0D010EF324D96E010EF42091
:1028D000DA6EDF50E56F29500E0D020EF324D96E2B
:1028E000010EF420DA6EDF50E66F29500E0D030E54
:1028F000F324D96E010EF420DA6EDF50E76F295011
:102900000E0D040EF324D96E010EF420DA6EDF50A2
:10291000E86F29500E0D050EF324D96E010EF42038
:10292000DA6EDF50E96F29500E0D060EF324D96ED2
:10293000010EF420DA6EDF50EA6F0B0E306EE00EFF
:102940001F6E30C020F0000E73EC19F0276E295076
:10295000750FD96EDA6ADF2A27C01AF00101E75134
:1029600099EC1DF0120028C0E0F024C0E1F02F0E19
:102970000001E26F000EE36F040E306EE00E1F6E7A
:1029800030C020F0000E73EC19F0276E3E8827C08F
:102990001AF00101E75199EC1DF0120028C0E0F097
:1029A00024C0E1F02E0E0001E26F000EE36F000E76
:1029B000E46F050E306E080E3E6EE0C0BAF0E1C066
:1029C000B9F0E2C0B8F0E3C0B7F0E00E1F6E30C05F
:1029D00020F0000E73EC19F0276E27C01AF00101E9
:1029E000E75199EC1DF012002550210AD8B44DD7BB
:1029F0000F0AD8B4D3D7010AD8A41200B4D70F6EE7
:102A00000BC001F00F5079EC1CF0106E0C9CAFD095
:102A10000FC0E0F00BC0E1F0210E0001E26F3104C5
:102A2000D8B4E28D0DC0E3F0000EE46F050E306EF9
:102A30000F0E1018D8B446D0230E016E105084EC3F
:102A40000EF0060E0001E46F10500E0D010EF3247F
:102A5000D96E010EF420DA6EDF50E56F10500E0DC6
:102A6000020EF324D96E010EF420DA6EDF50E66F09
:102A700010500E0D030EF324D96E010EF420DA6E01
:102A8000DF50E76F10500E0D040EF324D96E010EC7
:102A9000F420DA6EDF50E86F10500E0D050EF324AF
:102AA000D96E010EF420DA6EDF50E96F10500E0D72
:102AB000060EF324D96E010EF420DA6EDF50EA6FB1
:102AC0000B0E306EE00E066E30C007F0000EA4EC68
:102AD00019F00E6E1050750FD96EDA6ADF2A0EC02B
:102AE00001F00101E751AAEC1DF012000FC0E0F067
:102AF0000BC0E1F02F0E0001E26F000EE36F040E39
:102B0000306EE00E066E30C007F0000EA4EC19F037
:102B10000E6E3E880EC001F00101E751AAEC1DF0D7
:102B200012000FC0E0F00BC0E1F02E0E0001E26FCA
:102B3000000EE36F000EE46F050E306E080E3E6E61
:102B4000E0C0BAF0E1C0B9F0E2C0B8F0E3C0B7F05D
:102B5000E00E066E30C007F0000EA4EC19F00E6E09
:102B60000EC001F00101E751AAEC1DF012000C505B
:102B7000210AD8B44DD70F0AD8B4D3D7010AD8A4A4
:102B80001200B4D7256E25509F0FD96EDA6ADF5038
:102B90000001E06F25508D0FD96EDA6ADF50E16FCA
:102BA000210EE26F3104D8B4E28DBA0E2524D96E1D
:102BB000DA6A010EDA22DF50E36F230E1A6E255017
:102BC000BCEC0CF0060E0001E46F25500E0D010E5A
:102BD000F324D96E010EF420DA6EDF50E56F255034
:102BE0000E0D020EF324D96E010EF420DA6EDF50C2
:102BF000E66F25500E0D030EF324D96E010EF4205E
:102C0000DA6EDF50E76F25500E0D040EF324D96EF7
:102C1000010EF420DA6EDF50E86F25500E0D050E20
:102C2000F324D96E010EF420DA6EDF50E96F2550DF
:102C30000E0D060EF324D96E010EF420DA6EDF506D
:102C4000EA6F0B0E306EE00E1F6E30C020F0000EEB
:102C500073EC19F0246E2550750FD96EDA6ADF2AED
:102C600024C01AF00101E75199EC1DF02550810FA5
:102C7000D96EDA6A000EDF6E12000C6E0C509F0FD8
:102C8000D96EDA6ADF500001E06F0C508D0FD96EFB
:102C9000DA6ADF50E16F210EE26F3104D8B4E28DC1
:102CA000BA0E0C24D96EDA6A010EDA22DF50E36F15
:102CB000230E016E0C5084EC0EF0060E0001E46F42
:102CC0000C500E0D010EF324D96E010EF420DA6EB5
:102CD000DF50E56F0C500E0D020EF324D96E010E7D
:102CE000F420DA6EDF50E66F0C500E0D030EF32465
:102CF000D96E010EF420DA6EDF50E76F0C500E0D26
:102D0000040EF324D96E010EF420DA6EDF50E86F62
:102D10000C500E0D050EF324D96E010EF420DA6E60
:102D2000DF50E96F0C500E0D060EF324D96E010E24
:102D3000F420DA6EDF50EA6F0B0E306EE00E066E96
:102D400030C007F0000EA4EC19F00B6E0C50750F9C
:102D5000D96EDA6ADF2A0BC001F00101E751AAEC53
:102D60001DF00C50810FD96EDA6A000EDF6E120072
:102D7000F86FF5C01FF0F6C020F0070EA3EC1BF0B3
:102D80000001F851020F09EC1EF0010E1A6E3A0E06
:102D9000A7EC1AF0010E1A6E4C0EA7EC1AF0000107
:102DA000EF518DEC17F0300E4418D8B406D0010E58
:102DB0001A6E4450A7EC1AF005D0010E1A6E200EC0
:102DC000A7EC1AF0010E1A6E4350A7EC1AF000019E
:102DD000F0A506D0010E1A6E520EA7EC1AF005D01F
:102DE000010E1A6E560EA7EC1AF00001F039E846F3
:102DF0001F0B8DEC17F0300E4418D8B406D0010E1E
:102E00001A6E4450A7EC1AF005D0010E1A6E200E6F
:102E1000A7EC1AF0010E1A6E4350A7EC1AF000014D
:102E2000F451D8B408D0F5C01EF0100E1F6E210E5C
:102E30005EEC1BF01200F5C01EF0100E1F6E200E8F
:102E40005EEC1BF01200000E0101E66F000EE56F54
:102E5000FF0E2114236E070E2214246E23C01AF0D5
:102E600024C01BF0030E1D6EE80E1C6E56EC1AF00B
:102E70001AC0A7F01BC0A8F0A7C01AF0A8C01BF08A
:102E8000FC0E1D6E180E1C6E50EC1DF023501A2403
:102E9000236E24501B20246E23C01AF024C01BF084
:102EA000000E1D6E640E1C6E56EC1AF01AC0A5F0D2
:102EB0001BC0A6F0A5C01AF0A6C01BF0FF0E1D6E29
:102EC0009C0E1C6E50EC1DF023501A24236E2450CF
:102ED0001B20246E23C01AF024C01BF0000E1D6EB0
:102EE0000A0E1C6E56EC1AF01AC02CF01BC02DF006
:102EF0002CC01AF02DC01BF0FF0E1D6EF60E1C6EBE
:102F000050EC1DF023501A24236E24501B20246EF5
:102F100023C02AF024C02BF01200EE6F640E1A6E4C
:102F20000001EE5126EC1DF0446E0A0E1A6E44505C
:102F300026EC1DF0436E4350445C206E216AD8A0FD
:102F40002106000E236E0A0E226E17EC18F0205098
:102F5000446E44C01AF01B6AFF0E1D6EF60E1C6E06
:102F600050EC1DF00001EE51286E296A1A502826F7
:102F70001B5029224350285C206E2950D8A02904D8
:102F8000216E000E236E640E226E17EC18F0205096
:102F9000456E4550300F456E4450300F446E4350DF
:102FA000300F436E12000F0E296E35D063516CEC5A
:102FB00007F0296E0F0E2918D8B434D02950750F98
:102FC000D96EDA6ADF50D8B405D02950750FD96EA2
:102FD000DA6ADF062950750FD96EDA6ADF50D8B485
:102FE00005D02950750FD96EDA6ADF062950750FA2
:102FF000D96EDA6ADF50D8B405D02950750FD96E72
:10300000DA6ADF06C60E2924D96EDA6A010EDA22E0
:10301000000EDF6E07D06151400AD8B403D0C10A58
:10302000D8B4C4D7000E0001D76F29501200000E8B
:10303000256E23AE06D0226C231ED8B0232A010EA3
:10304000256E21AE06D0206C211ED8B0212A010E9B
:10305000251A000E276E000E266E22502310D8B4BB
:103060001CD0010E246E04D0D89022362336242A98
:1030700023AEFAD7D890263627362250205C23502C
:103080002158D8A005D02250205E2350215A2680F6
:10309000D89023322232242EEDD72550D8B404D034
:1030A000266C271ED8B0272A26C020F027C021F082
:1030B0001200590EF66E3C0EF76E000EF86E090007
:1030C000F5CFFDF00900F5CFFEF00900F5CFFFF0D8
:1030D000560EF66E3C0EF76E000EF86E0900F5CF38
:1030E00043F00900F5CF44F00900F5CF45F002EEBA
:1030F00000F0900EEE6AE806FDE101EE00F0FC0E35
:10310000EE6AE806FDE100EE60F08E0EEE6AE8067B
:10311000FDE100EE2AF0190EEE6AE806FDE14690A8
:103120004692000EF86E000132EF0AF0000E1E6E9D
:103130001E50990FD96EDA6A000EDF6EC60E1E247D
:10314000D96EDA6A010EDA22010EDF6E1E509F0F71
:10315000D96EDA6A1E50480FDF6E1E50580FF2EC1F
:103160001DF05A0AD8A409D01E508D0FD96EDA6A04
:103170001E50480FF2EC1DF005D01E508D0FD96E79
:10318000DA6A000EDF6E1E2A040E1E64D1D7010E0D
:10319000F2EC1DF00C0AD8B412000C0E1A6E010EDF
:1031A00040EC1CF01200010E1A6E020E2CEC1AF00C
:1031B0002A0E286E8E0EE82EFED7282EFCD7020E81
:1031C0001E6E010E05EC1CF05F0E1E6E0E0E1F6EC5
:1031D00002EC1AF0030E1E6E020E05EC1CF0A80E97
:1031E0001E6E090E1F6E02EC1AF0010E1A6E310EE1
:1031F000A7EC1AF0010E1A6E2E0EA7EC1AF0010EB3
:103200001A6E320EA7EC1AF034A21200010E1A6EDA
:10321000690EA7EC1AF01200000EB46E010E000148
:10322000D86F9CA202D09C989C8882824050600FEC
:10323000D96EDA6A98CFDFFF402A140E406402D0BC
:10324000000E406E030E4018D8B462C042F04050E9
:10325000016E026A4250036E046A040E0326000ED9
:103260000422015003180BE102500418D8A407D01F
:10327000010ED76F000ED86F40C0D4F01200000EC0
:10328000D76F1200000E826E000E836E000E846EE9
:10329000FC0E876E000E886E1A0E896EE00E0F010E
:1032A0001C6F1469FC0E0C6F000E286F000E136F5C
:1032B000010E0B6F000E1B6F000E0A6F000E126FD7
:1032C000000E1A6F096911691969090E0E01F26F72
:1032D000110EB06F140EB36F0D0EF56F0E0EF66F6C
:1032E000130EB26F1200226E020E0101E76F22C0B0
:1032F000E8F120C0E9F1000E236E0DD01F50232409
:10330000D96EDA6AEA0E2324E16EE26A010EE22245
:10331000DFCFE7FF232A2050235CD8A0EFD7E70EAA
:103320001A6E010E1B6E2350020F1C6E11EC1DF065
:10333000216EEA0E2324D96EDA6A010EDA2221C048
:10334000DFFF2350030F1200096E020E0101E76F29
:1033500009C0E8F107C0E9F1000E0A6E0DD0065071
:103360000A24D96EDA6AEA0E0A24E16EE26A010ED4
:10337000E222DFCFE7FF0A2A07500A5CD8A0EFD786
:10338000E70E016E010E026E0A50020F036E3BEC57
:103390001DF0086EEA0E0A24D96EDA6A010EDA22EE
:1033A00008C0DFFF0A50030F1200EF6F0001EF515A
:1033B0008DEC17F0300E4518D8A406D0010E1A6E09
:1033C000200EA7EC1AF005D0010E1A6E4550A7EC9E
:1033D0001AF0300E4518D8A40AD0300E4418D8A4DC
:1033E00006D0010E1A6E200EA7EC1AF005D0010EC1
:1033F0001A6E4450A7EC1AF0010E1A6E4350A7EC57
:103400001AF01200000E276E0ED0010E1A6E1E501A
:103410002724206E20C0F6FF080EF76E0800F55036
:10342000A7EC1AF0272AFF0E206EFF0E216E1F5008
:10343000226E236A20502226215023222750246EF8
:10344000256A2250245C2550800A266E2350800A6B
:103450002658D8B01200D9D71B6E1A04D8A41DD094
:10346000B60E00D000D0E82EFCD700D000D000D09F
:10347000849C8868000E1D6E849A848C848E8DCF07
:103480001CF0849E1CBE02D01D0E1D6E1D2A1D0E3A
:103490001D64F2D7849C000E886E000E886E849C9A
:1034A000849A1BC083FF848E849E1200000E206EBF
:1034B000000E1F6E1C501D10D8B41CD0010E1E6EC5
:1034C00004D0D8901C361D361E2A1DAEFAD7D890CF
:1034D0001F3620361C501A5C1D501B58D8A005D032
:1034E0001C501A5E1D501B5A1F80D8901D321C3272
:1034F0001E2EEDD71FC01AF020C01BF01200C09B7B
:10350000180E1A6E320E1B6E1BEC1EF0C099940E34
:103510001A6E390E1B6E16EC1EF0080E9E6E900E83
:103520009C6E240E9D6E8A0E9A6E000E9B6E000E8F
:10353000416E000E0001D36F000E3F6E000E406E14
:10354000000ED26F000ED16F0E01C08B12001B6EE9
:103550001A04D8A41DD0B60E00D000D0E82EFCD797
:1035600000D000D000D0849C8868000E1D6E849A24
:10357000848C848E8DCF1CF0849E1CBE02D01D0EC8
:103580001D6E1D2A1D0E1D64F2D7849C000E886ED0
:10359000849C848A1BC083FF848E849E1200000E4C
:1035A000656E000E666E000E676E000E686E000E91
:1035B000636E000E646E000E616E000E0F015A6F96
:1035C000000E586F000E546F000E556F000E566FB0
:1035D000000E606E000E536F000E516F000E526FA2
:1035E000940E5B6F000E576F12000E01C9A31200FC
:1035F0000001B129D8A403D0000EB16F01D0B12BC6
:10360000B051D8A4B007AF51D8A4AF07AE51D8A4D9
:10361000AE07AD51D8A4AD07CD51D8A4CD07AC515C
:10362000D8A4AC07AB51D8A4AB070E01C9931200C4
:10363000010E1A6E020E2CEC1AF02A0E286E8E0E57
:10364000E82EFED7282EFCD7010E1E6E010E05ECCB
:103650001CF0500E1E6E0F0E1F6E02EC1AF0010EC3
:103660001E6E020E05EC1CF0120E1E6E110E1F6E69
:1036700002EC1AF01200F26F0001F005D8B404D089
:10368000020EF019D8A41200F007F151D8B41200BC
:10369000110EF1611200F107F051400DF350800F4F
:1036A000F36FF351F125F36F010E1A6EF3512CEC09
:1036B0001AF00001F251D5EC19F01200206E1E0430
:1036C000D8B404D0020E1E18D8A412001E061F5033
:1036D000D8B41200110E1F6012001F061E50400DBC
:1036E000F350800F216E21501F24216E010E1A6E9F
:1036F00021502CEC1AF0010E1A6E2050A7EC1AF093
:10370000120032C022F03950D8B408D03250D8A4B8
:1037100002D0010E01D0000E326E02D0000E226ED9
:103720002250D8B408D0020E1E6E020E1F6E2A0E52
:103730005EEC1BF01200020E1E6E020E1F6E200EBB
:103740005EEC1BF01200216E1F04D8B404D0020EF0
:103750001F18D8A412001F062050D8B41200110E52
:103760002060120020061F50400DF350800F226E83
:1037700022502024226E010E1A6E22502CEC1AF0D8
:10378000215009EC1EF01200256E25C026F0276A94
:1037900026C021F027C022F023EC17F02C502D106A
:1037A000D8A406D0010E1A6E200EA7EC1AF006D08F
:1037B000010E1A6E2C50300FA7EC1AF0010E1A6E83
:1037C0002A50300FA7EC1AF012000F0E206E000ED8
:1037D000216E21509D08D96EDA6ADF50D8A40FD02F
:1037E000000E1D6E2150040823EC1CF0000E1D6E0F
:1037F0002150140823EC1CF021500408206E212ACB
:10380000030E2164E6D720501200206E2004D8B4A5
:1038100004D0020E2018D8A4120020061E50D8B4DE
:103820001200110E1E6012001E062050400DF350B3
:10383000800F1F6E1F501E241F6E010E1A6E1F5028
:103840002CEC1AF012001E6E1E50480F1F6E1F50F7
:10385000100FF2EC1DF05A0AD8B406D05A0E1A6EA8
:103860001F50100F40EC1CF01F50F2EC1DF01D1803
:10387000D8B412001DC01AF01F5040EC1CF012000A
:103880001B6E000EF2BE010E1C6E1BC079FF000EF7
:103890007A6E310E7B6E1AC07CFF7F8EF29E550EC3
:1038A000816EAA0E816E808880B8FED71CB002D0CF
:1038B000F29E01D0F28E7F9E12001C6E0F0E1D6EC6
:1038C000010E1E6E1E509F0FD96EDA6A1C50DE1854
:1038D000D8A409D01E508D0FD96EDA6A1A50DE189E
:1038E000D8B41EC01DF01E2A040E1E64EBD71D5056
:1038F0001200036E0F0E046E010E056E05509F0F31
:10390000D96EDA6A0350DE18D8A409D005508D0F9D
:10391000D96EDA6A0150DE18D8B405C004F0052A61
:10392000040E0564EBD7045012000F0E1A6E000E41
:103930001B6E1B509D08D96EDA6ADF50D8A40AD0DE
:103940001B509108D96EDA6ADF50D8A403D01B50FF
:1039500004081A6E1B2A030E1B64EBD71A501200C0
:103960003650170DF3CF25F0F4CF26F025C01AF00E
:1039700026C01BF0000E1D6E1E0E1C6E56EC1AF0BB
:103980001A50256E266A25C021F026C022F023ECAD
:1039900017F012003F50D8B40FD0E70E4124D96E73
:1039A000DA6A010EDA22DF50996E412A140E416460
:1039B00009D0150E416E06D0C099000E0001D66FD9
:1039C000000E406E3F0612001E6E1D50F2EC1DF000
:1039D0001E18D8B405D01EC01AF01D5040EC1CF0C3
:1039E0001D04F2EC1DF05A0AD8B412005A0E1A6ED9
:1039F0001D0440EC1CF01200010EB86E000EB76EF4
:103A0000000EB96EB568000EB46E0E01C997C1877D
:103A1000000E1A6E000E1B6E11EC1EF0D00EB66E6C
:103A20001200000E1D6E000E1E6E0AD01E501A24CB
:103A3000D96E000E1B20DA6EDF501D181D6E1E2A77
:103A40001E501C5CD8B0F2D71D5012001B6E080E21
:103A50001C6E000E1D6ED8901B341D341D6ED89048
:103A60001B361A501D5CD8A002D01A501D5E1C2EA9
:103A7000F2D71D501200000E046E000E056E0AD023
:103A800005500124D96E000E0220DA6EDF500418B2
:103A9000046E052A0550035CD8B0F2D7045012001A
:103AA0001A501C02F3CF1EF0F4CF1FF01A501D0263
:103AB000F3501F261B501C02F3501F261EC01AF085
:103AC0001FC01BF012001E6E1EC05AFF0F015B8F3D
:103AD0005B9D5B815BB1FED75F511D6E1C6A5E51C1
:103AE0001C241A6E000E1D201B6E1200010E1A6E91
:103AF000010E2CEC1AF0290E1F6E960E1E6E7F0E14
:103B0000E82EFED71E2EFCD71F2EFAD700F012008B
:103B100029EC1EF0CBEC1DF042EC19F0FEEC1DF090
:103B2000CFEC1AF0FCEC1CF0D9EC1DF07FEC1AF095
:103B300012001B6E010E0001D66F1AC0D5F01AC01C
:103B40003FF00E01C0B904D01BC099FF010E416EB9
:103B5000C0891200026E010E0001D66F01C0D5F0BF
:103B600001C03FF00E01C0B904D002C099FF010EA0
:103B7000416EC0891200000E946E260E956E010EE5
:103B8000966E400E976EF00E936E900E926E0E0132
:103B9000C891C0811200000E0E01DC6F000EDD6FB7
:103BA000000EDE6F000EDF6F000EE06F000EE16FA3
:103BB0001200050EBE6E000EBD6E000EBF6EBB681D
:103BC000000EBA6EC993A00EBC6E120095EC1CF0EC
:103BD000226E0F0E2218D8A403D0E5EC1BF0226E43
:103BE000225012001A6E1AC079FF000E7A6E310E42
:103BF0007B6E808000F000F07C501200600ED36F6E
:103C0000000ED56F000ED76F080ED96F000ED86F5B
:103C100012001E6E010E1A6E1E50300FA7EC1AF025
:103C200012001AC0A4F21BC0A5F212001AC0FEF1C5
:103C30001BC0FFF112001AC0FCF11BC0FDF1120005
:103C4000C997000E406E82921200B68E1200BC8E92
:103C50001200F29A12002020200E2020FFFFFFFF0A
:103C6000FFFFFFFFFFFFFFFFFFFFFFFFFFFFFFFF64
:103C7000FFFFFFFFFFFFFFFFFFFFFFFFFFFFFFFF54
:103C8000FFFFFFFFFFFFFFFFFFFFFFFFFFFFFFFF44
:103C9000FFFFFFFFFFFFFFFFFFFFFFFFFFFFFFFF34
:020000040030CA
:0C0000008CFFFFFF9FFFFFFEFFFFFFFFD4
:020000040020DA
:10000000FFFFFFFFFFFFFFFFFFFFFFFFFFFFFFFF00
:10001000FFFFFFFFFFFFFFFFFFFFFFFFFFFFFFFFF0
:10002000FFFFFFFFFFFFFFFFFFFFFFFFFFFFFFFFE0
:10003000FFFFFFFFFFFFFFFFFFFFFFFFFFFFFFFFD0
:10004000FFFFFFFFFFFFFFFFFFFFFFFFFFFFFFFFC0
:10005000FFFFFFFFFFFFFFFFFFFFFFFFFFFFFFFFB0
:10006000FFFFFFFFFFFFFFFFFFFFFFFFFFFFFFFFA0
:10007000FFFFFFFFFFFFFFFFFFFFFFFFFFFFFFFF90
:10008000FFFFFFFFFFFFFFFFFFFFFFFFFFFFFFFF80
:10009000FFFFFFFFFFFFFFFFFFFFFFFFFFFFFFFF70
:1000A000FFFFFFFFFFFFFFFFFFFFFFFFFFFFFFFF60
:1000B000FFFFFFFFFFFFFFFFFFFFFFFFFFFFFFFF50
:1000C000FFFFFFFFFFFFFFFFFFFFFFFFFFFFFFFF40
:1000D000FFFFFFFFFFFFFFFFFFFFFFFFFFFFFFFF30
:1000E000FFFFFFFFFFFFFFFFFFFFFFFFFFFFFFFF20
:1000F000FFFFFFFFFFFFFFFFFFFFFFFFFFFFFFFF10
:020000040031C9
:10000000FF0CFFFFFFFFFFFFFFFFFFFFFFFFFFFFF3
:10001000FFFFFFFFFFFFFFFFFFFFFFFFFFFFFFFFF0
:10002000FFFFFFFFFFFFFFFFFFFFFFFFFFFFFFFFE0
:10003000FFFFFFFFFFFFFFFFFFFFFFFFFFFFFFFFD0
:10004000FFFFFFFFFFFFFFFFFFFFFFFFFFFFFFFFC0
:10005000FFFFFFFFFFFFFFFFFFFFFFFFFFFFFFFFB0
:10006000FFFFFFFFFFFFFFFFFFFFFFFFFFFFFFFFA0
:10007000FFFFFFFFFFFFFFFFFFFFFFFFFFFFFFFF90
:10008000FFFFFFFFFFFFFFFFFFFFFFFFFFFFFFFF80
:10009000FFFFFFFFFFFFFFFFFFFFFFFFFFFFFFFF70
:1000A000FFFFFFFFFFFFFFFFFFFFFFFFFFFFFFFF60
:1000B000FFFFFFFFFFFFFFFFFFFFFFFFFFFFFFFF50
:1000C000FFFFFFFFFFFFFFFFFFFFFFFFFFFFFFFF40
:1000D000FFFFFFFFFFFFFFFFFFFFFFFFFFFFFFFF30
:1000E000FFFFFFFFFFFFFFFFFFFFFFFFFFFFFFFF20
:1000F000FFFFFFFFFFFFFFFFFFFFFFFFFFFFFFFF10
:00000001FF
